:020000040000FA
:0A00000000000000A4EF00F0B4D0EF
:0800180001D1126E960E096E73
:10002000980E0A6E6AD8D8B4CA90D8A4CA80FC0FB9
:10003000D8A0CA92D8B0CA82800E096E960E0A6EF7
:10004000980E0D6E0E6ACAB025D8CAB223D857D8FA
:100050000904CB6E09C00BF00AC00CF000500F6E03
:10006000106E003C106A60D80E50122E0AD0BE6E80
:100070000C0EBD6E0DBEBD8A0DBCBD889394CA84A6
:100080001200BB6E0C0EBA6E0DBEBA8A0DBCBA88D9
:100090009492F5D700D8D8900D320A320932120066
:1000A000E836E836FC0B0109C212C009C216C0507E
:1000B000F80B0309C06E320E15D8C282C2B2FED749
:1000C000C4CF16F0C350156E12000C6A0B6EFF0EF3
:1000D0000B260C2200D0D8A01200030E0A6EE60EEA
:1000E00002D8F5D70A6AFE0F096EE86A0A5AD8A044
:1000F00012000000090600D0F8D70E6A0D6A100E33
:10010000F36E0A340D360E360B500D5C0C500E5843
:1001100005E30B500D5E0C500E5AD88009360A3696
:10012000F32EEFD7095012000B500F02F3CF0DF052
:10013000F4CF0EF00C500F02F3500E260B501002AD
:10014000F3500E260D5012004F0EAF6E240EAC6E03
:10015000900EAB6E0001C69A430E926EE00E936E47
:10016000C00E946E8A0EC06E0E0EC16E010EC26E6F
:10017000C2D0F2A403D0F294817A11009EAA19D0C1
:10018000060EAB1412E1E2CF4AF0E1CF49F04B2A60
:1001900010EE4EF04B50E126000EE222AECFE7FF0C
:1001A0004AC0E2FF49C0E1FF1100AE50AE50AB982B
:1001B000AB8811004B504C5C14E04C2AEACF0AF09B
:1001C000E9CF09F000EE4EF04C50E926000EEA228D
:1001D000EF50096E0AC0EAFF09C0E9FFD88012009B
:1001E00004D0E868096ED8A0120012004B6A4C6A6D
:1001F0009D8A9F8AF28EF28C12009D9A00EE4EF03C
:10020000010EF46EF36AF306000EF45AEE6AF4502F
:10021000F310F9E14B6A4C6A9D8A1200F29EC2CF3C
:100220004EF1C1CF4FF1C0CF50F1C4CF51F1C3CF88
:1002300052F1E0CF53F109C054F10AC055F10FC09B
:1002400056F111C057F115C058F116C059F1D8CF69
:100250005AF1E8CF5BF1F28E0001A192B30EB36EBA
:10026000D40EB26E000E1CDF396E16C03AF0395053
:1002700037263A503822D89038323732010E385C5F
:100280006E0ED8B4375C04E2010E386E6E0E376E17
:10029000020E385C08E303E1510E375C04E3020E02
:1002A000386E500E376E00016E0E375C3C6E8270F9
:1002B000F29E4EC1C2FF4FC1C1FF50C1C0FF51C12C
:1002C000C4FF52C1C3FF53C1E0FF54C109F055C17F
:1002D0000AF056C10FF057C111F058C115F059C1BD
:1002E00016F05AC1D8FF5BC1E8FFF28E10009EA83D
:1002F000FED7AD6E12009294899492968986939A55
:100300008A9A006A4C0E0C6E500E0B6E020E85DE41
:1003100094948B9494968B9693948A94336A466AB9
:10032000456A446A0A0E306E316A6E0E326E3D6A5C
:1003300030C03FF0D8903234406E939A8A8A0A0EC9
:10034000C4DE939A8A9A52DF58DFCD6AF294F28A19
:10035000870ED56E000EA4DE376E16C038F0010E83
:10036000385C6E0ED8B4375C04E2010E386E6E0E47
:10037000376E020E385C08E303E1510E375C04E38C
:10038000020E386E500E376E00016E0E375C3C6EFA
:100390003CC03BF0B16AA192A082B36AB26AD08E2F
:1003A000A292B10EB16E06DF1D6EC00E1D5C07E39A
:1003B000FE0E1D5C02E396D002D01F6A93D01DAEE4
:1003C00021D01F6A8F0E1D5C05E11DC01FF0206843
:1003D000216817D09F0E1D5C05E11DC01FF022682B
:1003E00023680FD0AF0E1D5C05E11DC01FF024680F
:1003F000256807D0BF0E1D5C04E11DC01FF02668F4
:10040000276870D01F5202E16DD06CD08F0E1F5C38
:1004100014E1202803E11DC020F00DD01DC021F003
:10042000220E205C07E35C0E205C04E24552D8A457
:1004300045064D80206856D055D09F0E1F5C39E18F
:10044000222803E11DC022F032D01DC023F0235228
:100450000DE1220E225C07E35C0E225C04E24552B1
:10046000D8A445064D8022683DD020D0220E225CC3
:100470001DE35C0E225C1AE2166A45C015F0455079
:100480001526000E162245501526000E1622186A53
:1004900022C017F0210E175E000E185A15501724AF
:1004A000456ED8904532D89045324D9022681AD08A
:1004B00019D0AF0E1F5C0AE1242803E11DC024F00F
:1004C00002D01DC025F024680DD00CD0BF0E1F5CDB
:1004D00009E1262803E11DC026F003D01DC027F046
:1004E000E2D800D0D7CF1AF0D6CF19F03E501AB4C8
:1004F0000108D8B4D0D03E6A1AB43E2A46A00AD029
:10050000D89045343D6ED8903D36E30E3D5C02E315
:10051000E20E3D6E3C503B5C0CE13C503D5C06E025
:100520004D82FD0E445CD8A0442A02D0446A4D920C
:1005300007D03CC03BF04D92020E445CD8B044065C
:10054000FF0E3D24016E026AFF0E0222025205E1F7
:1005500001503C5C02E13DC03CF0026A3D28016E66
:10056000D8B4022A025205E101503C5C02E13DC0D0
:100570003CF0036A046A026AD8903C30D890E832B2
:10058000016E076A086A066AD8903D30D890E83252
:10059000056E0550015C1EE10650025C1BE1075030
:1005A000035C18E10850045C15E1E86A80A6010FBD
:1005B000D8B48094D8A48084006A4C0E0C6E500E7F
:1005C0000B6E020E0DEC00F08B948B968A84400E1D
:1005D000476E5CD0076A086A066AD8903D30D890AA
:1005E000E832056E0150055C02500658035007586A
:1005F000045008582CE27F0E475CD8B4446A8986C0
:1006000089845F0E3C5C06E23C505F08416ED890E6
:10061000413203D05F0E3C5C416E436A44C042F0FD
:10062000435203E14250405C03E2436A40C042F05F
:10063000000142C000F04C0E0C6E500E0B6E020E0C
:100640000DEC00F08B948A948B86476A1FD047523A
:10065000D8B4446A89968994436A44C042F04352AC
:1006600003E14250405C03E2436A40C042F00001B3
:1006700042C000F04C0E0C6E500E0B6E020E0DECD4
:1006800000F08B848B968A947F0E476E4DA003D02A
:100690004552D8A44506827886D6286812002A6872
:1006A000120029681200150E265C0AE127C030F0FE
:1006B0007C0E305C02E37B0E306E30C03FF046D0E3
:1006C000160E265C12E133A00BD027C031F0D89073
:1006D00031343D6EE30E3D5C02E3E20E3D6E01D02F
:1006E0003D6AD8903D30316E31D0170E265C0EE158
:1006F00027C032F0D8903234406E40503F5C02E365
:100700003F28406ED8904030326E20D0420E265C9A
:1007100009E1275203E133901BD803D033803D6AAF
:10072000316A14D0430E265C0BE133A008D027C0F9
:1007300046F0275202E0468002D04690456A06D035
:100740007B0E265C03E1456A3D6A316A2668120029
:100750003C520FE13D6A006A4C0E0C6E500E0B6E5F
:10076000020E0DEC00F0898489968B968B948A8416
:1007700001D03D6A0A0E306E316A6E0E326E30C0A4
:100780003FF0D8903230406E466A456A469012007B
:02079000FFD791
:020000040030CA
:0300010006170ED1
:020005008580F4
:060008000FC00FE00F40E5
:00000001FF
